:020000040000FA
:0408000070EF09F09C
:1008100003B284EF05F0F2B4A2EF05F09EB0AAEFA8
:1008200005F09EB2B2EF05F0F2A81AEF04F0F2B2B2
:1008300032EF04F09EB61FEF04F01FEF09F09E9612
:1008400000011550000A06E000011550010A06E0FB
:100850001FEF09F021EC21F01FEF09F019EC23F054
:100860001FEF09F0CD90F2929EA03CEF04F0010141
:10087000533F3CEF04F0542BB2C1B6F1B3C1B7F112
:10088000B4C1B8F1B5C1B9F1AEC1B2F1AFC1B3F104
:10089000B0C1B4F1B1C1B5F1AAC1AEF1ABC1AFF114
:1008A000ACC1B0F1ADC1B1F1A6C1AAF1A7C1ABF124
:1008B000A8C1ACF1A9C1ADF1A2C1A6F1A3C1A7F134
:1008C000A4C1A8F1A5C1A9F19EC1A2F19FC1A3F144
:1008D000A0C1A4F1A1C1A5F19AC19EF19BC19FF154
:1008E0009CC1A0F19DC1A1F1CECF9AF1CFCF9BF1D8
:1008F00053C19CF154C19DF1CF6ACE6A0101536B83
:10090000546B9E90CD800FBC0F8E0FBA8BEF04F00E
:100910000F8A1FEF09F013880F8C0FBEC8EF04F089
:100920009AC19EF19BC19FF19CC1A0F19DC1A1F113
:100930009EC1A2F19FC1A3F1A0C1A4F1A1C1A5F1E3
:10094000A2C1A6F1A3C1A7F1A4C1A8F1A5C1A9F1B3
:10095000A6C1AAF1A7C1ABF1A8C1ACF1A9C1ADF183
:10096000AAC1AEF1ABC1AFF1ACC1B0F1ADC1B1F153
:10097000AEC1B2F1AFC1B3F1B0C1B4F1B1C1B5F123
:10098000B2C1B6F1B3C1B7F1B4C1B8F1B5C1B9F1F3
:1009900001015E6B5F6B606B616B9A515E279B51CF
:1009A0005F239C5160239D5161239E515E279F517F
:1009B0005F23A0516023A1516123A2515E27A3515F
:1009C0005F23A4516023A5516123A6515E27A7513F
:1009D0005F23A8516023A9516123AA515E27AB511F
:1009E0005F23AC516023AD516123AE515E27AF51FF
:1009F0005F23B0516023B1516123B2515E27B351DF
:100A00005F23B4516023B5516123B6515E27B751BE
:100A10005F23B8516023B9516123D890010161333C
:100A200060335F335E33D8900101613360335F33ED
:100A30005E33D8900101613360335F335E3300C1B0
:100A40000CF101C10DF102C10EF103C10FF104C19E
:100A500010F105C111F106C112F107C113F108C16E
:100A600014F109C115F10AC116F10BC117F134C116
:100A700035F111B847EF05F00101620E046F010E68
:100A8000056F000E066F000E076F50EF05F00101B5
:100A9000A70E046F020E056F000E066F000E076FA3
:100AA0005EC100F15FC101F160C102F161C103F1FA
:100AB000B8EC1FF003BF04D01ABE02D01AA0108CED
:100AC00011A068EF05F010BA68EF05F00F80108AEA
:100AD0000CC100F10DC101F10EC102F10FC103F112
:100AE00010C104F111C105F112C106F113C107F1E2
:100AF00014C108F115C109F116C10AF117C10BF1B2
:100B000035C134F11FEF09F00392ABB2AB98AB885B
:100B1000030103EE00F080517F0BE92604C0EFFFD4
:100B2000802B8151805D700BD8A48B820000805196
:100B3000815D700BD8A48B9281518019D8B4079035
:100B40001FEF09F0F2940101453F1FEF09F0462B1A
:100B50001FEF09F09E900101533F1FEF09F0542B46
:100B60001FEF09F09E9211B827EF07F08BB4C0EF8A
:100B700005F010ACC0EF05F08B84109CC1EF05F0C0
:100B80008B94C3CF55F1C4CF56F1C28207B430EF76
:100B900006F047C14BF148C14CF149C14DF14AC182
:100BA0004EF15EC162F15FC163F160C164F161C188
:100BB00065F113A8DEEF05F0138C13989AC1BAF112
:100BC0009BC1BBF19CC1BCF19DC1BDF19EC1BEF1F9
:100BD0009FC1BFF1A0C1C0F1A1C1C1F1A2C1C2F1C9
:100BE000A3C1C3F1A4C1C4F1A5C1C5F1A6C1C6F199
:100BF000A7C1C7F1A8C1C8F1A9C1C9F1AAC1CAF169
:100C0000ABC1CBF1ACC1CCF1ADC1CDF1AEC1CEF138
:100C1000AFC1CFF1B0C1D0F1B1C1D1F1B2C1D2F108
:100C2000B3C1D3F1B4C1D4F1B5C1D5F1B6C1D6F1D8
:100C3000B7C1D7F1B8C1D8F1B9C1D9F10101555146
:100C40005B2756515C23E86A5D230E2E30EF06F0D9
:100C50005CC157F15DC158F15B6B5C6B5D6B078EDE
:100C60000201002F1FEF09F03C0E006F1B50E00B3C
:100C7000E00AE866128819BE02D019B4108E00C1CD
:100C80000CF101C10DF102C10EF103C10FF104C15C
:100C900010F105C111F106C112F107C113F108C12C
:100CA00014F109C115F10AC116F10BC117F134C1D4
:100CB00035F101018E6764EF06F08F6764EF06F08F
:100CC000906764EF06F0916768EF06F098EF06F022
:100CD00092C100F193C101F194C102F195C103F1F8
:100CE0000101010E046F000E056F000E066F000E6D
:100CF000076FB8EC1FF000C192F101C193F102C17E
:100D000094F103C195F100678DEF06F001678DEF57
:100D100006F002678DEF06F0036798EF06F08EC1CC
:100D200092F18FC193F190C194F191C195F10F802F
:100D3000D57ED5BE6ED0D6CF47F1D7CF48F145C1CD
:100D400049F1E86AE8CF4AF1138A1ABE02D01AA024
:100D5000108C109047C100F148C101F149C102F166
:100D60004AC103F101010A0E046F000E056F000E67
:100D7000066F000E076FB8EC1FF003AF1080010183
:100D800054A7CFEF06F00F9A0F9C0F9E0101000EA3
:100D90005E6F600E5F6F3D0E606F080E616F010148
:100DA00047BFDFEF06F04867DFEF06F04967DFEF88
:100DB00006F04A67DFEF06F0F28804EF07F0F298DA
:100DC0005E6B5F6B606B616B9A6B9B6B9C6B9D6BDF
:100DD0009E6B9F6BA06BA16BA26BA36BA46BA56BAF
:100DE000A66BA76BA86BA96BAA6BAB6BAC6BAD6B5F
:100DF000AE6BAF6BB06BB16BB26BB36BB46BB56B0F
:100E0000B66BB76BB86BB96BD76AD66A0101456B25
:100E1000466B0CC100F10DC101F10EC102F10FC111
:100E200003F110C104F111C105F112C106F113C1A2
:100E300007F114C108F115C109F116C10AF117C172
:100E40000BF135C134F11FEF09F01FEF09F002017A
:100E5000002F81EF08F0D59ED6CF47F1D7CF48F1CC
:100E600045C149F1E86AE8CF4AF1138AD76AD66AE0
:100E70000101456B466BD58E1B50E00BE00AE8661E
:100E8000128819BE02D019B4108E18AE1D8C00C184
:100E90000CF101C10DF102C10EF103C10FF104C14A
:100EA00010F105C111F106C112F107C113F108C11A
:100EB00014F109C115F10AC116F10BC117F134C1C2
:100EC00035F10FA0109A11B871EF07F00101620E11
:100ED000046F010E056F000E066F000E076F7AEFAC
:100EE00007F00101A70E046F020E056F000E066FDA
:100EF000000E076F47C100F148C101F149C102F17D
:100F00004AC103F1B8EC1FF003BF8DEF07F01ABE22
:100F100002D01AA0108C11B00F800CC100F10DC1CD
:100F200001F10EC102F10FC103F110C104F111C1B1
:100F300005F112C106F113C107F114C108F115C181
:100F400009F116C10AF117C10BF135C134F10201E3
:100F50003C0E006F00C10CF101C10DF102C10EF198
:100F600003C10FF104C110F105C111F106C112F165
:100F700007C113F108C114F109C115F10AC116F135
:100F80000BC117F134C135F101018E67CFEF07F0C6
:100F90008F67CFEF07F09067CFEF07F09167D3EF40
:100FA00007F003EF08F092C100F193C101F194C181
:100FB00002F195C103F10101010E046F000E056FEE
:100FC000000E066F000E076FB8EC1FF000C192F123
:100FD00001C193F102C194F103C195F10067F8EFEB
:100FE00007F00167F8EF07F00267F8EF07F0036713
:100FF00003EF08F08EC192F18FC193F190C194F18B
:1010000091C195F10F80109047C100F148C101F1E5
:1010100049C102F14AC103F101010A0E046F000E39
:10102000056F000E066F000E076FB8EC1FF003AFE0
:101030001080010154A729EF08F00F9A0F9C0F9E12
:101040000101000E5E6F600E5F6F3D0E606F080E57
:10105000616F47C100F148C101F149C102F14AC1C4
:1010600003F10101140E046F050E056F000E066FEB
:10107000000E076FB8EC1FF003AF42EF08F0F288E4
:1010800067EF08F0F2985E6B5F6B606B616B9A6B59
:101090009B6B9C6B9D6B9E6B9F6BA06BA16BA26B04
:1010A000A36BA46BA56BA66BA76BA86BA96BAA6BB4
:1010B000AB6BAC6BAD6BAE6BAF6BB06BB16BB26B64
:1010C000B36BB46BB56BB66BB76BB86BB96B0CC16C
:1010D00000F10DC101F10EC102F10FC103F110C108
:1010E00004F111C105F112C106F113C107F114C1D8
:1010F00008F115C109F116C10AF117C10BF135C18B
:1011000034F1D8EC23F01E661ED01DAE11D01D9E0A
:101110001E8E19AE07D0156A040E166E176A21ECE2
:1011200021F011D0156A166A176A21EC21F00BD054
:101130001DAC09D01D9C1E8C010E156E166A176A17
:1011400019EC23F000D08BB4ADEF08F010ACADEF8C
:1011500008F08B84109CAEEF08F08B94C3CF55F150
:10116000C4CF56F1C28207B41DEF09F047C14BF15D
:1011700048C14CF149C14DF14AC14EF15EC162F125
:101180005FC163F160C164F161C165F113A8CBEF88
:1011900008F0138C13989AC1BAF19BC1BBF19CC1A2
:1011A000BCF19DC1BDF19EC1BEF19FC1BFF1A0C107
:1011B000C0F1A1C1C1F1A2C1C2F1A3C1C3F1A4C1D7
:1011C000C4F1A5C1C5F1A6C1C6F1A7C1C7F1A8C1A7
:1011D000C8F1A9C1C9F1AAC1CAF1ABC1CBF1ACC177
:1011E000CCF1ADC1CDF1AEC1CEF1AFC1CFF1B0C147
:1011F000D0F1B1C1D1F1B2C1D2F1B3C1D3F1B4C117
:10120000D4F1B5C1D5F1B6C1D6F1B7C1D7F1B8C1E6
:10121000D8F1B9C1D9F1010155515B2756515C2371
:10122000E86A5D230E2E1DEF09F05CC157F15DC128
:1012300058F15B6B5C6B5D6B078E1FEF09F002C0B2
:10124000E0FF005001C0D8FF1000A6B225EF09F062
:101250000CC0A9FF0BC0A8FFA69EA69CA684F29E68
:10126000550EA76EAA0EA76EA682F28EA694A6B2FF
:1012700037EF09F00C2A1200A96EA69EA69CA68044
:10128000A8500C2A120004012C0E826F4DEC0BF0BA
:10129000B3EC20F00C503CEC09F0E8CF00F10C501E
:1012A0003CEC09F0E8CF01F101AF5CEF09F001017E
:1012B000FF0E026FFF0E036F56EC20F0296768EFF8
:1012C00009F00401200E826F4DEC0BF06DEF09F078
:1012D00004012D0E826F4DEC0BF060EC1EF012003D
:1012E000316A076A0F6A106A116A126A136A0F017B
:1012F0000E0EC16E860EC06E030EC26E0F01896A9D
:10130000110E926E080E8A6EF10E936E8B6A980E15
:10131000946EF18EFC0E3CEC09F0E8CF0BF00BA0C4
:1013200011800BA211820BA411840BA81188C90E85
:101330003CEC09F0E8CF18F0CA0E3CEC09F0E8CF1D
:1013400019F0CB0E3CEC09F0E8CF1AF0CC0E3CECD7
:1013500009F0E8CF1BF0CE0E3CEC09F0E8CF14F01A
:10136000CD0E3CEC09F0E8CF30F01D6A1E6A0E6A23
:1013700001015B6B5C6B5D6B576B586BF29A010103
:10138000476B486B496B4A6B4B6B4C6B4D6B4E6BB1
:101390004F6B506B516B526B456B466BD76AD66A7D
:1013A0000F01280ED56EF28A9D90B00ECD6E010110
:1013B0005E6B5F6B606B616B626B636B646B656BC9
:1013C000666B676B686B696B536B546BCF6ACE6AE5
:1013D0000F9A0F9C0F9E9D80760ECA6E9D82020111
:1013E0003C0E006FCC6A160E3CEC09F0E8CF00F121
:1013F000170E3CEC09F0E8CF01F1180E3CEC09F0B7
:10140000E8CF02F1190E3CEC09F0E8CF03F101013D
:1014100003AF25EF0AF0B3EC20F0160E0C6E00C1FE
:101420000BF025EC09F0170E0C6E01C10BF025EC4A
:1014300009F0180E0C6E02C10BF025EC09F0190E24
:101440000C6E03C10BF025EC09F000C18EF101C157
:101450008FF102C190F103C191F100C192F101C17C
:1014600093F102C194F103C195F11A0E3CEC09F01D
:10147000E8CF00F11B0E3CEC09F0E8CF01F11C0EA7
:101480003CEC09F0E8CF02F11D0E3CEC09F0E8CF8E
:1014900003F1010103AF7BEF0AF0B3EC20F01A0E69
:1014A0000C6E00C10BF025EC09F01B0E0C6E01C197
:1014B0000BF025EC09F01C0E0C6E02C10BF025ECB4
:1014C00009F01D0E0C6E03C10BF025EC09F01A0E8D
:1014D0003CEC09F0E8CF00F11B0E3CEC09F0E8CF42
:1014E00001F11C0E3CEC09F0E8CF02F11D0E3CECC2
:1014F00009F0E8CF03F100C196F101C197F102C1F3
:1015000098F103C199F1240EAC6E900EAB6E240ECF
:10151000AC6E080EB86E000EB06E1F0EAF6E0401FA
:10152000806B816B0F01900EAB6E0F019D8A0301E2
:10153000806B816BC26B8B92156A166A176A9D86E7
:1015400007900001F28EF28C07B009EF1DF00FB08A
:101550001CEF16F010BE1CEF16F012B81CEF16F0C0
:101560000301805181197F0BD8B409EF1DF013EEF0
:1015700000F081517F0BE126812BE7CFE8FFE00BE4
:10158000D8B409EF1DF023EE82F0C2513F0BD926EB
:10159000E7CFDFFFC22BDF50780AD8A409EF1DF098
:1015A000078092C100F193C101F194C102F195C18C
:1015B00003F10101040E046F000E056F000E066FAB
:1015C000000E076FB8EC1FF000AFF0EF0AF001015A
:1015D000030E926F000E936F000E946F000E956FC6
:1015E00003018251720AD8B4F8EF15F08251520A01
:1015F000D8B4F8EF15F08251750AD8B4F8EF15F0A9
:101600008251630AD8B4C3EF19F08251690AD8B481
:101610009AEF12F082517A0AD8B4ADEF13F08251EA
:10162000490AD8B439EF12F08251500AD8B443EFC6
:1016300011F08251700AD8B48BEF11F08251540A24
:10164000D8B4BBEF11F08251740AD8B406EF12F08F
:101650008251410AD8B463EF0CF082514B0AD8B4DE
:1016600061EF0BF082516D0AD8B496EF10F0825101
:101670004D0AD8B4AFEF10F08251730AD8B428EFF6
:1016800015F08251530AD8B48DEF15F08251590AE2
:10169000D8B4E7EF0FF0FAEF19F0040114EE00F000
:1016A00080517F0BE12682C4E7FF802B12000401EA
:1016B0000D0E826F4DEC0BF00A0E826F4DEC0BF0AD
:1016C000120004014B0E826F4DEC0BF004012C0E46
:1016D000826F4DEC0BF081B802D030B630D00301F0
:1016E0008351430AD8B4A6EF0BF003018351630A78
:1016F000D8B4A8EF0BF003018351520AD8B4AAEF73
:101700000BF003018351720AD8B4ACEF0BF0030164
:101710008351470AD8B4AEEF0BF003018351670A37
:10172000D8B4B0EF0BF003018351540AD8B4B2EF30
:101730000BF003018351740AD8B421EF0CF00301BC
:101740008351550AD8B4B4EF0BF082D030807AD0F0
:10175000309078D0308276D0309274D0308472D08D
:10176000309470D030866ED084C330F185C331F1AF
:1017700086C332F187C333F10101296B01EC21F0FB
:1017800078EC20F000C104F101C105F102C106F1BD
:1017900003C107F1F4EC20F0200EF86EF76AF66A48
:1017A0000900F5CF2CF10900F5CF2DF10900F5CF97
:1017B0002EF10900F5CF2FF10900F5CF30F1090026
:1017C000F5CF31F10900F5CF32F10900F5CF33F152
:1017D0000101296B01EC21F078EC20F0B8EC1FF04E
:1017E0000067FAEF0BF00167FAEF0BF00267FAEF10
:1017F0000BF0036701D025D004014E0E826F4DEC33
:101800000BF004016F0E826F4DEC0BF004014D0ED6
:10181000826F4DEC0BF00401610E826F4DEC0BF00A
:101820000401740E826F4DEC0BF00401630E826FA5
:101830004DEC0BF00401680E826F4DEC0BF0F8EFED
:1018400019F03096CD0E0C6E30C00BF025EC09F07F
:10185000CD0E3CEC09F0E8CF30F030B006D00401FA
:10186000630E826F4DEC0BF005D00401430E826FC6
:101870004DEC0BF030B206D00401720E826F4DECCD
:101880000BF005D00401520E826F4DEC0BF030B41A
:1018900006D00401670E826F4DEC0BF005D00401F9
:1018A000470E826F4DEC0BF030B606D00401740E7B
:1018B000826F4DEC0BF005D00401540E826F4DEC9D
:1018C0000BF0F8EF19F00401410E826F4DEC0BF0B4
:1018D00003018351310AD8B407EF0FF0030183519C
:1018E000320AD8B437EF0EF003018351330AD8B46B
:1018F000C0EF0DF003018351340AD8B4B0EF0CF0FF
:1019000003018351350AD8B48DEF0CF004013F0E6A
:10191000826F4DEC0BF0F8EF19F004012C0E826F82
:101920004DEC0BF003018451300AD8B4A0EF0CF059
:1019300003018451310AD8B4A8EF0CF0F9EF0DF08F
:101940008B900401300E826F4DEC0BF0AEEF0CF07B
:101950008B800401310E826F4DEC0BF0F8EF19F023
:10196000CC0E3CEC09F0E8CF0BF004012C0E826F9A
:101970004DEC0BF003018451310AD8B4D4EF0CF0D4
:1019800003018451300AD8B4D6EF0CF0030184511E
:101990004D0AD8B4E0EF0CF003018451540AD8B4D6
:1019A000E7EF0CF0FEEF0CF08A8401D08A940BAEC6
:1019B00004D00BAC02D00BBA21D0E00E0B1218D021
:1019C0001F0E0B168539E844E00B0B1211D0E00E08
:1019D0000B16F4EC20F085C332F186C333F101011C
:1019E000296B01EC21F078EC20F000511F0B0B1259
:1019F000CC0E0C6E0BC00BF025EC09F00401340E7C
:101A0000826F4DEC0BF004012C0E826F4DEC0BF04D
:101A1000CC0E3CEC09F0E8CF1BF08AB406D00401F0
:101A2000300E826F4DEC0BF005D00401310E826F49
:101A30004DEC0BF004012C0E826F4DEC0BF01B38BB
:101A4000E840070BE8CF82F40401300E82274DEC0A
:101A50000BF004012C0E826F4DEC0BF0B3EC20F078
:101A60001B501F0BE8CF00F156EC20F032C182F47E
:101A70000401300E82274DEC0BF033C182F40401D7
:101A8000300E82274DEC0BF004012C0E826F4DECD2
:101A90000BF0B3EC20F02EC000F100AF0BD0FF0E26
:101AA000016FFF0E026FFF0E036F04012D0E826F98
:101AB0004DEC0BF056EC20F031C182F40401300EF5
:101AC00082274DEC0BF032C182F40401300E8227E4
:101AD0004DEC0BF033C182F40401300E82274DEC43
:101AE0000BF004012C0E826F4DEC0BF0B3EC20F0E8
:101AF0002DC000F156EC20F031C182F40401300E0B
:101B000082274DEC0BF032C182F40401300E8227A3
:101B10004DEC0BF033C182F40401300E82274DEC02
:101B20000BF004012C0E826F4DEC0BF0B3EC20F0A7
:101B30002FC000F100AF0BD0FF0E016FFF0E026F40
:101B4000FF0E036F04012D0E826F4DEC0BF056EC6F
:101B500020F031C182F40401300E82274DEC0BF0ED
:101B600032C182F40401300E82274DEC0BF033C1F8
:101B700082F40401300E82274DEC0BF0F8EF19F0DF
:101B8000CB0E3CEC09F0E8CF0BF004012C0E826F79
:101B90004DEC0BF003018451450AD8B4E4EF0DF08D
:101BA00003018451440AD8B4E7EF0DF003018451D6
:101BB000300AD8B4EAEF0DF003018451310AD8B4E9
:101BC000EEEF0DF0F9EF0DF00B9EF3EF0DF00B8E35
:101BD000F3EF0DF0FC0E0B16F3EF0DF0FC0E0B16F1
:101BE0000B80F3EF0DF0CB0E0C6E0BC00BF025EC61
:101BF00009F00401330E826F4DEC0BF004012C0E42
:101C0000826F4DEC0BF0CB0E3CEC09F0E8CF1AF0F4
:101C10001ABE12EF0EF00401450E826F4DEC0BF070
:101C200017EF0EF00401440E826F4DEC0BF004012F
:101C30002C0E826F4DEC0BF00401300E826F4DECD8
:101C40000BF004012C0E826F4DEC0BF01AB030EF4C
:101C50000EF00401300E826F4DEC0BF035EF0EF0FC
:101C60000401310E826F4DEC0BF0F8EF19F0CA0E43
:101C70003CEC09F0E8CF0BF004012C0E826F4DEC28
:101C80000BF003018451450AD8B473EF0EF0030141
:101C90008451440AD8B476EF0EF0030184514D0A02
:101CA000D8B47FEF0EF003018451410AD8B479EF24
:101CB0000EF003018451460AD8B47CEF0EF0030104
:101CC0008451560AD8B487EF0EF003018451500AAC
:101CD000D8B492EF0EF003018451520AD8B495EFB4
:101CE0000EF09EEF0EF00B9E98EF0EF00B8E98EF1D
:101CF0000EF00B9C98EF0EF00B8C98EF0EF0FC0E94
:101D00000B1685C3E8FF030B0B1298EF0EF0C70EFE
:101D10000B1685C3E8FF070BE846E846E8460B12BA
:101D200098EF0EF00B8498EF0EF00B9498EF0EF0F6
:101D3000CA0E0C6E0BC00BF025EC09F0CA0E3CEC81
:101D400009F0E8CF19F00401320E826F4DEC0BF070
:101D500004012C0E826F4DEC0BF019BEB7EF0EF0A4
:101D60000401450E826F4DEC0BF0BCEF0EF0040148
:101D7000440E826F4DEC0BF004012C0E826F4DEC83
:101D80000BF019C0E8FF030BE8CF82F40401300E1A
:101D900082274DEC0BF004012C0E826F4DEC0BF002
:101DA00019BCDAEF0EF00401410E826F4DEC0BF01E
:101DB000DFEF0EF00401460E826F4DEC0BF00401D4
:101DC0002C0E826F4DEC0BF019C0E8FF380BE84287
:101DD000E842E842E8CF82F40401300E82274DEC5D
:101DE0000BF004012C0E826F4DEC0BF019B400EFD8
:101DF0000FF00401520E826F4DEC0BF005EF0FF067
:101E00000401500E826F4DEC0BF0F8EF19F0C90E83
:101E10003CEC09F0E8CF0BF004012C0E826F4DEC86
:101E20000BF003018451450AD8B425EF0FF00301EC
:101E30008451440AD8B428EF0FF0030184514D0AAD
:101E4000D8B42BEF0FF039EF0FF00B9E33EF0FF0FC
:101E50000B8E33EF0FF0F80E0B1685C3E8FF070B60
:101E60000B1233EF0FF0C90E0C6E0BC00BF025EC0C
:101E700009F00401310E826F4DEC0BF004012C0EC1
:101E8000826F4DEC0BF0C90E3CEC09F0E8CF18F076
:101E900018BE06D00401450E826F4DEC0BF005D044
:101EA0000401440E826F4DEC0BF004012C0E826F86
:101EB0004DEC0BF018C0E8FF070BE8CF82F40401EB
:101EC000300E82274DEC0BF004012C0E826F4DEC8E
:101ED0000BF00780B3EC20F029C0E8FF003B004383
:101EE0000043030B56EC20F033C182F40401300EA2
:101EF00082274DEC0BF004012C0E826F4DEC0BF0A1
:101F0000B3EC20F029C001F1019F019D2AC000F12E
:101F1000010156EC20F02FC182F40401300E82271B
:101F20004DEC0BF030C182F40401300E82274DECF1
:101F30000BF031C182F40401300E82274DEC0BF01E
:101F400032C182F40401300E82274DEC0BF033C114
:101F500082F40401300E82274DEC0BF004012C0EAC
:101F6000826F4DEC0BF0B3EC20F02BC001F12CC0D4
:101F700000F1D89001330033D890013300330101D0
:101F800056EC20F02FC182F40401300E82274DEC74
:101F90000BF030C182F40401300E82274DEC0BF0BF
:101FA00031C182F40401300E82274DEC0BF032C1B6
:101FB00082F40401300E82274DEC0BF033C182F421
:101FC0000401300E82274DEC0BF0F8EF19F0FC0EF7
:101FD0003CEC09F0E8CF0BF003018351520AD8B46E
:101FE0001EEF10F003018351720AD8B421EF10F0F4
:101FF00003018351500AD8B424EF10F00301835138
:10200000700AD8B427EF10F003018351550AD8B4F1
:102010002AEF10F003018351750AD8B42DEF10F0A8
:1020200003018351430AD8B436EF10F00301835102
:10203000630AD8B439EF10F042EF10F00B903CEF88
:1020400010F00B803CEF10F00B923CEF10F00B8285
:102050003CEF10F00B943CEF10F00B843CEF10F0D1
:102060000B963CEF10F00B863CEF10F00B983CEF1A
:1020700010F00B883CEF10F0FC0E0C6E0BC00BF058
:1020800025EC09F00401590E826F4DEC0BF0119014
:10209000119211941198FC0E3CEC09F0E8CF0BF072
:1020A0000BA011800BA211820BA411840BA8118824
:1020B00011A062EF10F00401520E826F4DEC0BF094
:1020C00067EF10F00401720E826F4DEC0BF011A857
:1020D00071EF10F00401430E826F4DEC0BF076EFC0
:1020E00010F00401630E826F4DEC0BF011A280EF33
:1020F00010F00401500E826F4DEC0BF085EF10F0E4
:102100000401700E826F4DEC0BF011A48FEF10F0F4
:102110000401550E826F4DEC0BF094EF10F00401AA
:10212000750E826F4DEC0BF0F8EF19F004016D0E97
:10213000826F4DEC0BF003018351300AD8B4F3EFFA
:1021400010F003018351310AD8B406EF11F00301F6
:102150008351320AD8B419EF11F0FAEF19F081B8AF
:1021600003D030B4F8EF19F004014D0E826F4DEC3E
:102170000BF0F4EC20F084C331F185C332F186C357
:1021800033F10101296B01EC21F078EC20F003011F
:102190008351300AD8B4DBEF10F003018351310AC8
:1021A000D8B4E3EF10F003018351320AD8B4EBEF57
:1021B00010F0FAEF19F0FD0E0C6E00C10BF025ECDB
:1021C00009F0F3EF10F0FE0E0C6E00C10BF025ECE1
:1021D00009F006EF11F0FF0E0C6E00C10BF025ECBC
:1021E00009F019EF11F00401300E826F4DEC0BF085
:1021F00004012C0E826F4DEC0BF0B3EC20F0FD0EC1
:102200003CEC09F0E8CF00F12AEF11F00401310EA7
:10221000826F4DEC0BF004012C0E826F4DEC0BF035
:10222000B3EC20F0FE0E3CEC09F0E8CF00F12AEF11
:1022300011F00401320E826F4DEC0BF0B3EC20F084
:1022400004012C0E826F4DEC0BF0FF0E3CEC09F0FC
:10225000E8CF00F156EC20F031C182F40401300ED9
:1022600082274DEC0BF032C182F40401300E82273C
:102270004DEC0BF033C182F40401300E82274DEC9B
:102280000BF0F8EF19F081B803D030B239EF12F04B
:1022900083C32AF184C32BF185C32CF186C32DF1AE
:1022A00087C32EF188C32FF189C330F18AC331F17E
:1022B0008BC332F18CC333F1010101EC21F078ECD6
:1022C00020F0160E0C6E00C10BF025EC09F0170E75
:1022D0000C6E01C10BF025EC09F0180E0C6E02C15A
:1022E0000BF025EC09F0190E0C6E03C10BF025EC78
:1022F00009F000C18EF101C18FF102C190F103C15B
:1023000091F100C192F101C193F102C194F103C1B5
:1023100095F139EF12F081B803D030B239EF12F0F5
:1023200083C32AF184C32BF185C32CF186C32DF11D
:1023300087C32EF188C32FF189C330F18AC331F1ED
:102340008BC332F18CC333F1010101EC21F078EC45
:1023500020F000C18EF101C18FF102C190F103C1E3
:1023600091F100C192F101C193F102C194F103C155
:1023700095F139EF12F081B803D030B239EF12F095
:1023800083C32AF184C32BF185C32CF186C32DF1BD
:1023900087C32EF188C32FF189C330F18AC331F18D
:1023A0008CC332F18DC333F1010101EC21F078ECE3
:1023B00020F00101000E046F000E056F010E066F84
:1023C000000E076FC9EC1FF01A0E0C6E00C10BF067
:1023D00025EC09F01B0E0C6E01C10BF025EC09F089
:1023E0001C0E0C6E02C10BF025EC09F01D0E0C6EDC
:1023F00003C10BF025EC09F000C196F101C197F182
:1024000002C198F103C199F139EF12F081B803D0FC
:1024100030B239EF12F083C32AF184C32BF185C3A4
:102420002CF186C32DF187C32EF188C32FF189C308
:1024300030F18AC331F18CC332F18DC333F1010124
:1024400001EC21F078EC20F00101000E046F000E89
:10245000056F010E066F000E076FC9EC1FF000C17B
:1024600096F101C197F102C198F103C199F139EFD9
:1024700012F0160E3CEC09F0E8CF00F1170E3CEC20
:1024800009F0E8CF01F1180E3CEC09F0E8CF02F1B9
:10249000190E3CEC09F0E8CF03F156EC20F019ECF2
:1024A0001EF00401730E826F4DEC0BF004012C0E34
:1024B000826F4DEC0BF08EC100F18FC101F190C124
:1024C00002F191C103F156EC20F019EC1EF0040169
:1024D000730E826F4DEC0BF004012C0E826F4DECED
:1024E0000BF01A0E3CEC09F0E8CF00F11B0E3CECAF
:1024F00009F0E8CF01F11C0E3CEC09F0E8CF02F145
:102500001D0E3CEC09F0E8CF03F115EC1AF00401C4
:102510002C0E826F4DEC0BF096C100F197C101F1CA
:1025200098C102F199C103F115EC1AF057EC0BF0C8
:10253000FAEF19F00401690E826F4DEC0BF0040103
:102540002C0E826F4DEC0BF00101040E006F000E9B
:10255000016F000E026F000E036F56EC20F02CC1CD
:1025600082F40401300E82274DEC0BF02DC182F471
:102570000401300E82274DEC0BF02EC182F40401D1
:10258000300E82274DEC0BF02FC182F40401300E87
:1025900082274DEC0BF030C182F40401300E82270B
:1025A0004DEC0BF031C182F40401300E82274DEC6A
:1025B0000BF032C182F40401300E82274DEC0BF097
:1025C00033C182F40401300E82274DEC0BF004017C
:1025D0002C0E826F4DEC0BF00101030E006F000E0C
:1025E000016F000E026F000E036F56EC20F02CC13D
:1025F00082F40401300E82274DEC0BF02DC182F4E1
:102600000401300E82274DEC0BF02EC182F4040140
:10261000300E82274DEC0BF02FC182F40401300EF6
:1026200082274DEC0BF030C182F40401300E82277A
:102630004DEC0BF031C182F40401300E82274DECD9
:102640000BF032C182F40401300E82274DEC0BF006
:1026500033C182F40401300E82274DEC0BF00401EB
:102660002C0E826F4DEC0BF001013B0E006F000E43
:10267000016F000E026F000E036F56EC20F02CC1AC
:1026800082F40401300E82274DEC0BF02DC182F450
:102690000401300E82274DEC0BF02EC182F40401B0
:1026A000300E82274DEC0BF02FC182F40401300E66
:1026B00082274DEC0BF030C182F40401300E8227EA
:1026C0004DEC0BF031C182F40401300E82274DEC49
:1026D0000BF032C182F40401300E82274DEC0BF076
:1026E00033C182F40401300E82274DEC0BF004015B
:1026F0002C0E826F4DEC0BF0200EF86EF76AF66A26
:1027000004010900F5CF82F44DEC0BF00900F5CF80
:1027100082F44DEC0BF00900F5CF82F44DEC0BF098
:102720000900F5CF82F44DEC0BF00900F5CF82F4EF
:102730004DEC0BF00900F5CF82F44DEC0BF00900E5
:10274000F5CF82F44DEC0BF00900F5CF82F44DEC9F
:102750000BF057EC0BF0FAEF19F081B803D030B062
:10276000FDEF13F08351630AD8A4F8EF19F08451F8
:10277000610AD8A4F8EF19F085516C0AD8A4F8EFD3
:1027800019F08651410A42E08651440A1BE0865105
:10279000420AD8B419EF14F08651350AD8B484EF40
:1027A0001BF08651360AD8B4D9EF1BF08651370A90
:1027B000D8B442EF1CF08651380AD8B4A0EF1CF010
:1027C000F8EF19F00798079A04017A0E826F4DEC22
:1027D0000BF00401780E826F4DEC0BF00401640ED7
:1027E000826F4DEC0BF081A8FDEF13F00401550E44
:1027F000826F4DEC0BF002EF14F004014C0E826F6F
:102800004DEC0BF057EC0BF0FAEF19F00788079A34
:1028100004017A0E826F4DEC0BF00401410E826FC1
:102820004DEC0BF00401610E826F4DEC0BF0F3EFF9
:1028300013F00798078A04017A0E826F4DEC0BF0B3
:102840000401420E826F4DEC0BF00401610E826FA9
:102850004DEC0BF0F3EF13F00101666737EF14F066
:10286000676737EF14F0686737EF14F0696715D0C2
:102870004F6742EF14F0506742EF14F0516742EF98
:1028800014F052670AD00101000E006F000E016FB4
:10289000000E026F000E036F120011B80AD0010182
:1028A000620E046F010E056F000E066F000E076FBB
:1028B00009D00101A70E046F020E056F000E066F0E
:1028C000000E076F66C100F167C101F168C102F136
:1028D00069C103F1B8EC1FF003BFDFEF14F0119AE8
:1028E000119C0101000E046FA80E056F550E066FB6
:1028F000020E076F66C100F167C101F168C102F104
:1029000069C103F166C18AF167C18BF168C18CF1BD
:1029100069C18DF1B8EC1FF003BF0BD00101000EAF
:102920008A6FA80E8B6F550E8C6F020E8D6F118AF9
:10293000119C0E0E3CEC09F0E8CF18F10F0E3CECA8
:1029400009F0E8CF19F1100E3CEC09F0E8CF1AF1CC
:10295000110E3CEC09F0E8CF1BF101EC1FF08AC12D
:1029600004F18BC105F18CC106F18DC107F1B8EC02
:102970001FF00782C5EC1EF001EC1FF00792C5ECBA
:102980001EF08AC100F18BC101F18CC102F18DC131
:1029900003F10792C5EC1EF0CC0E046FE00E056F3C
:1029A000870E066F050E076FB8EC1FF000C118F117
:1029B00001C119F102C11AF103C11BF140D013AAE0
:1029C000E4EF14F0138E139A119C119A0101800EFA
:1029D000006F1A0E016F060E026F000E036F4FC1DB
:1029E00004F150C105F151C106F152C107F1B8EC33
:1029F0001FF003AF05D0B3EC20F0118C119A120038
:102A00000E0E3CEC09F0E8CF18F10F0E3CEC09F08B
:102A1000E8CF19F1100E3CEC09F0E8CF1AF1110ED5
:102A20003CEC09F0E8CF1BF14FC100F150C101F1BE
:102A300051C102F152C103F10782C5EC1EF018C169
:102A400000F119C101F11AC102F11BC103F1120019
:102A50000401730E826F4DEC0BF004012C0E826F9B
:102A60004DEC0BF0078462C166F163C167F164C18C
:102A700068F165C169F14BC14FF14CC150F14DC1D5
:102A800051F14EC152F157C159F158C15AF1079451
:102A90004EEC15F057EC0BF0FAEF19F066C100F1AF
:102AA00067C101F168C102F169C103F1010156EC8E
:102AB00020F019EC1EF00401630E826F4DEC0BF058
:102AC00004012C0E826F4DEC0BF04FC100F150C190
:102AD00001F151C102F152C103F1010156EC20F0A4
:102AE00019EC1EF00401660E826F4DEC0BF0040130
:102AF0002C0E826F4DEC0BF0B3EC20F059C100F1BD
:102B00005AC101F1010156EC20F019EC1EF004014C
:102B1000740E826F4DEC0BF0120010820401530E04
:102B2000826F4DEC0BF004012C0E826F4DEC0BF01C
:102B300083C32AF184C32BF185C32CF186C32DF105
:102B400087C32EF188C32FF189C330F18AC331F1D5
:102B50008BC332F18CC333F1010101EC21F078EC2D
:102B600020F000C166F101C167F102C168F103C143
:102B700069F18EC32AF18FC32BF190C32CF191C35D
:102B80002DF192C32EF193C32FF194C330F195C36D
:102B900031F196C332F197C333F1010101EC21F019
:102BA00078EC20F000C14FF101C150F102C151F1A8
:102BB00003C152F1F4EC20F099C32FF19AC330F124
:102BC0009BC331F19CC332F19DC333F1010101EC90
:102BD00021F078EC20F000C159F101C15AF14EEC1E
:102BE00015F004012C0E826F4DEC0BF008EF16F07F
:102BF000118E1AA002D01AAE108C19BE02D019A4E0
:102C0000108E03018251520A02E10F8201D00F920D
:102C10008251750A02E1108401D010948251550A44
:102C200002E1108601D010968351310A03E113822C
:102C3000138402D01392139411A003D011A401D0D5
:102C40001084078410B286EF16F010A46AEF16F015
:102C5000BAC166F1BBC167F1BCC168F1BDC169F120
:102C6000BEC16AF1BFC16BF1C0C16CF1C1C16DF1F0
:102C7000C2C16EF1C3C16FF1C4C170F1C5C171F1C0
:102C8000C6C172F1C7C173F1C8C174F1C9C175F190
:102C9000CAC176F1CBC177F1CCC178F1CDC179F160
:102CA000CEC17AF1CFC17BF1D0C17CF1D1C17DF130
:102CB000D2C17EF1D3C17FF1D4C180F1D5C181F100
:102CC000D6C182F1D7C183F1D8C184F1D9C185F1D0
:102CD00072EF16F062C166F163C167F164C168F119
:102CE00065C169F1BAC186F1BBC187F1BCC188F188
:102CF000BDC189F14BC14FF14CC150F14DC151F1F2
:102D00004EC152F157C159F158C15AF107940FA061
:102D1000A8EF16F00101966795EF16F0976795EF0B
:102D200016F0986795EF16F0996799EF16F0A8EFEF
:102D300016F02CEC14F096C104F197C105F198C17E
:102D400006F199C107F1B8EC1FF003BFBEEF19F00F
:102D50002CEC14F00101000E046F000E056F010E43
:102D6000066F000E076FE9EC1FF011A02AD011A228
:102D700028D056EC20F0296701D005D004012D0E93
:102D8000826F4DEC0BF030C182F40401300E8227CB
:102D90004DEC0BF031C182F40401300E82274DEC72
:102DA0000BF032C182F40401300E82274DEC0BF09F
:102DB00033C182F40401300E82274DEC0BF057EC46
:102DC0000BF012A8C5D012981BC01CF01C3A1C4274
:102DD000070E1C1600011C50000AD8B474EF17F03F
:102DE00000011C50010AD8B400EF17F000011C507C
:102DF000020AD8B4FEEF16F0A6EF17F0A6EF17F010
:102E0000B3EC20F02BC001F12CC000F1D8900133BD
:102E10000033D890013300330101630E046F000EBC
:102E2000056F000E066F000E076FE9EC1FF0280E0D
:102E3000046F000E056F000E066F000E076FB8ECF2
:102E40001FF000C12EF0B3EC20F029C001F1019F6A
:102E5000019D2AC000F10101A40E046F000E056F50
:102E6000000E066F000E076FE9EC1FF000C12DF099
:102E700000C104F101C105F102C106F103C107F16E
:102E8000640E006F000E016F000E026F000E036FE4
:102E9000B8EC1FF0050E046F000E056F000E066FF4
:102EA000000E076FE9EC1FF000C104F101C105F14C
:102EB00002C106F103C107F1B3EC20F02EC000F10E
:102EC000B8EC1FF000C12FF02FC0E8FF050F2E5CFB
:102ED00003E78A84A6EF17F02FC0E8FF0A0F2E5CE5
:102EE00001E68A94A6EF17F000C124F101C125F193
:102EF00002C126F103C127F1B3EC20F0B9EC20F0B8
:102F00001B501F0BE8CF00F10101640E046F000E8F
:102F1000056F000E066F000E076FC9EC1FF024C18D
:102F200004F125C105F126C106F127C107F1B8EC6E
:102F30001FF003BF02D08A9401D08A8424C100F11B
:102F400025C101F126C102F127C103F1FAEF19F001
:102F500000C124F101C125F102C126F103C127F10D
:102F600010AE4DD0109E00C108F101C109F102C19F
:102F70000AF103C10BF156EC20F030C1DAF131C196
:102F8000DBF132C1DCF133C1DDF108C100F109C16F
:102F900001F10AC102F10BC103F101016C0E046FD2
:102FA000070E056F000E066F000E076FB8EC1FF0DE
:102FB00003BF04D00101550EDE6F1CD008C100F123
:102FC00009C101F10AC102F10BC103F10101A40E13
:102FD000046F060E056F000E066F000E076FB8EC4B
:102FE0001FF003BF04D001017F0EDE6F03D001018B
:102FF000FF0EDE6F1D8E11AEBEEF19F0119E24C1C3
:1030000000F125C101F126C102F127C103F111A090
:1030100005D011A203D00FB0BEEF19F010A418EF25
:1030200018F00401750E826F4DEC0BF01DEF18F0D7
:103030000401720E826F4DEC0BF004012C0E826FB6
:103040004DEC0BF056EC20F029672CEF18F0040142
:10305000200E826F2FEF18F004012D0E826F4DECC1
:103060000BF030C182F40401300E82274DEC0BF0DE
:1030700031C182F40401300E82274DEC0BF00401C3
:103080002E0E826F4DEC0BF032C182F40401300E33
:1030900082274DEC0BF033C182F40401300E8227FD
:1030A0004DEC0BF004016D0E826F4DEC0BF0040142
:1030B0002C0E826F4DEC0BF04FC100F150C101F1AD
:1030C00051C102F152C103F1010156EC20F019EC9B
:1030D0001EF00401480E826F4DEC0BF004017A0ED5
:1030E000826F4DEC0BF004012C0E826F4DEC0BF057
:1030F00066C100F167C101F168C102F169C103F164
:10310000010156EC20F019EC1EF00401630E826FF1
:103110004DEC0BF004012C0E826F4DEC0BF066C1F0
:1031200000F167C101F168C102F169C103F1010158
:103130000A0E046F000E056F000E066F000E076F7B
:10314000C9EC1FF0000E046F120E056F000E066F23
:10315000000E076FE9EC1FF056EC20F02AC182F454
:103160000401300E82274DEC0BF02BC182F40401D8
:10317000300E82274DEC0BF02CC182F40401300E8E
:1031800082274DEC0BF02DC182F40401300E822712
:103190004DEC0BF02EC182F40401300E82274DEC71
:1031A0000BF02FC182F40401300E82274DEC0BF09E
:1031B00030C182F40401300E82274DEC0BF0040183
:1031C0002E0E826F4DEC0BF031C182F40401300EF3
:1031D00082274DEC0BF032C182F40401300E8227BD
:1031E0004DEC0BF033C182F40401300E82274DEC1C
:1031F0000BF00401730E826F4DEC0BF004012C0EEA
:10320000826F4DEC0BF0B3EC20F059C100F15AC1C4
:1032100001F124EC1BF013A25DEF19F004012C0E58
:10322000826F4DEC0BF086C166F187C167F188C1F2
:1032300068F189C169F12CEC14F00101000E046FF2
:10324000000E056F010E066F000E076FE9EC1FF010
:1032500056EC20F0296732EF19F00401200E826F3E
:1032600035EF19F004012D0E826F4DEC0BF030C1DB
:1032700082F40401300E82274DEC0BF031C182F450
:103280000401300E82274DEC0BF004012E0E826FEC
:103290004DEC0BF032C182F40401300E82274DEC6C
:1032A0000BF033C182F40401300E82274DEC0BF099
:1032B00004016D0E826F4DEC0BF013A484EF19F036
:1032C00004012C0E826F4DEC0BF013AC72EF19F071
:1032D0000401500E826F4DEC0BF0139C1398139A5F
:1032E00084EF19F013AE7FEF19F00401460E826FE0
:1032F0004DEC0BF0139E1398139A84EF19F0040110
:10330000530E826F4DEC0BF00FB28AEF19F00FA045
:10331000BCEF19F004012C0E826F4DEC0BF0200E67
:10332000F86EF76AF66A04010900F5CF82F44DECF5
:103330000BF00900F5CF82F44DEC0BF00900F5CF4E
:1033400082F44DEC0BF00900F5CF82F44DEC0BF05C
:103350000900F5CF82F44DEC0BF00900F5CF82F4B3
:103360004DEC0BF00900F5CF82F44DEC0BF00900A9
:10337000F5CF82F44DEC0BF057EC0BF00F90109E54
:103380001298FAEF19F00401630E826F4DEC0BF006
:1033900004012C0E826F4DEC0BF000EC1AF00401CE
:1033A0002C0E826F4DEC0BF073EC1AF004012C0E16
:1033B000826F4DEC0BF0EFEC1AF004012C0E826FD3
:1033C0004DEC0BF00101F80E006FCD0E016F660E93
:1033D000026F030E036F15EC1AF004012C0E826FBE
:1033E0004DEC0BF005EC1BF057EC0BF0FAEF19F07D
:1033F00057EC0BF00301C26B0790109209EF1DF020
:10340000D8900E0E3CEC09F0E8CF00F10F0E3CEC2A
:1034100009F0E8CF01F1100E3CEC09F0E8CF02F121
:10342000110E3CEC09F0E8CF03F10101000E046F2E
:10343000000E056F010E066F000E076FE9EC1FF01E
:1034400056EC20F02AC182F40401300E82274DECA4
:103450000BF02BC182F40401300E82274DEC0BF0EF
:103460002CC182F40401300E82274DEC0BF02DC1EB
:1034700082F40401300E82274DEC0BF02EC182F451
:103480000401300E82274DEC0BF02FC182F40401B1
:10349000300E82274DEC0BF030C182F40401300E67
:1034A00082274DEC0BF031C182F40401300E8227EB
:1034B0004DEC0BF004012E0E826F4DEC0BF032C17F
:1034C00082F40401300E82274DEC0BF033C182F4FC
:1034D0000401300E82274DEC0BF004016D0E826F5B
:1034E0004DEC0BF01200120E3CEC09F0E8CF00F1AD
:1034F000130E3CEC09F0E8CF01F1140E3CEC09F09E
:10350000E8CF02F1150E3CEC09F0E8CF03F1010120
:103510000A0E046F000E056F000E066F000E076F97
:10352000C9EC1FF0000E046F120E056F000E066F3F
:10353000000E076FE9EC1FF056EC20F02AC182F470
:103540000401300E82274DEC0BF02BC182F40401F4
:10355000300E82274DEC0BF02CC182F40401300EAA
:1035600082274DEC0BF02DC182F40401300E82272E
:103570004DEC0BF02EC182F40401300E82274DEC8D
:103580000BF02FC182F40401300E82274DEC0BF0BA
:1035900030C182F40401300E82274DEC0BF004019F
:1035A0002E0E826F4DEC0BF031C182F40401300E0F
:1035B00082274DEC0BF032C182F40401300E8227D9
:1035C0004DEC0BF033C182F40401300E82274DEC38
:1035D0000BF00401730E826F4DEC0BF012000A0E1B
:1035E0003CEC09F0E8CF00F10B0E3CEC09F0E8CF21
:1035F00001F10C0E3CEC09F0E8CF02F10D0E3CECB1
:1036000009F0E8CF03F124EF1BF0060E3CEC09F0C3
:10361000E8CF00F1070E3CEC09F0E8CF01F1080E0D
:103620003CEC09F0E8CF02F1090E3CEC09F0E8CFE0
:1036300003F124EF1BF00101B3EC20F0078457C124
:1036400000F158C101F107940101E80E046F800EEA
:10365000056F000E066F000E076FC9EC1FF0000E1D
:10366000046F040E056F000E066F000E076FE9EC85
:103670001FF0880E046F130E056F000E066F000E0C
:10368000076FB8EC1FF00A0E046F000E056F000EF6
:10369000066F000E076FE9EC1FF056EC20F00101F9
:1036A000296758EF1BF00401200E826F5BEF1BF0BF
:1036B00004012D0E826F4DEC0BF030C182F4040139
:1036C000300E82274DEC0BF031C182F40401300E34
:1036D00082274DEC0BF032C182F40401300E8227B8
:1036E0004DEC0BF004012E0E826F4DEC0BF033C14C
:1036F00082F40401300E82274DEC0BF00401430EDE
:10370000826F4DEC0BF0120087C32AF188C32BF1B6
:1037100089C32CF18AC32DF18BC32EF18CC32FF1F9
:103720008DC330F18EC331F190C332F191C333F1C7
:103730000101296B01EC21F078EC20F00101000E71
:10374000046F000E056F010E066F000E076FC9ECC7
:103750001FF00E0E0C6E00C10BF025EC09F00F0EE1
:103760000C6E01C10BF025EC09F0100E0C6E02C1BD
:103770000BF025EC09F0110E0C6E03C10BF025ECDB
:1037800009F004017A0E826F4DEC0BF004012C0E4F
:10379000826F4DEC0BF00401350E826F4DEC0BF097
:1037A00004012C0E826F4DEC0BF000EC1AF002EFCE
:1037B00014F087C32AF188C32BF189C32CF18AC383
:1037C0002DF18BC32EF18CC32FF18DC330F18EC33D
:1037D00031F190C332F191C333F10101296B01EC56
:1037E00021F078EC20F0880E046F130E056F000EA8
:1037F000066F000E076FBDEC1FF0000E046F040E85
:10380000056F000E066F000E076FC9EC1FF0010177
:10381000E80E046F800E056F000E066F000E076F36
:10382000E9EC1FF00A0E0C6E00C10BF025EC09F05C
:103830000B0E0C6E01C10BF025EC09F00C0E0C6E9A
:1038400002C10BF025EC09F00D0E0C6E03C10BF05C
:1038500025EC09F004017A0E826F4DEC0BF00401A7
:103860002C0E826F4DEC0BF00401360E826F4DEC86
:103870000BF004012C0E826F4DEC0BF0EFEC1AF004
:1038800002EF14F087C32AF188C32BF189C32CF10E
:103890008AC32DF18BC32EF18CC32FF18DC330F170
:1038A0008FC331F190C332F191C333F1010101ECC7
:1038B00021F078EC20F0000E046F120E056F000E60
:1038C000066F000E076FC9EC1FF001010A0E046FAE
:1038D000000E056F000E066F000E076FE9EC1FF07B
:1038E000120E0C6E00C10BF025EC09F0130E0C6EDD
:1038F00001C10BF025EC09F0140E0C6E02C10BF0A7
:1039000025EC09F0150E0C6E03C10BF025EC09F047
:1039100004017A0E826F4DEC0BF004012C0E826FC5
:103920004DEC0BF00401370E826F4DEC0BF00401EF
:103930002C0E826F4DEC0BF073EC1AF002EF14F0CA
:1039400087C32AF188C32BF189C32CF18AC32DF1D7
:103950008BC32EF18CC32FF18DC330F18EC331F1A7
:1039600090C332F191C333F10101296B01EC21F0D5
:1039700078EC20F0880E046F130E056F000E066FB2
:10398000000E076FBDEC1FF0000E046F040E056FF4
:10399000000E066F000E076FC9EC1FF00101E80E64
:1039A000046F800E056F000E066F000E076FE9ECC6
:1039B0001FF0060E0C6E00C10BF025EC09F0070E8F
:1039C0000C6E01C10BF025EC09F0080E0C6E02C163
:1039D0000BF025EC09F0090E0C6E03C10BF025EC81
:1039E00009F004017A0E826F4DEC0BF004012C0EED
:1039F000826F4DEC0BF00401380E826F4DEC0BF032
:103A000004012C0E826F4DEC0BF005EC1BF002EF65
:103A100014F081B803D030B0C7EF1DF007A881EFD4
:103A20001DF00101800E006F1A0E016F060E026F6D
:103A3000000E036F4BC104F14CC105F14DC106F1FD
:103A40004EC107F1B8EC1FF003BFC7EF1DF013EC38
:103A50001EF04BC100F14CC101F14DC102F14EC14C
:103A600003F10782C5EC1EF018C104F119C105F17C
:103A70001AC106F11BC107F1F80E006FCD0E016FE0
:103A8000660E026F030E036FB8EC1FF00E0E0C6E85
:103A900000C10BF025EC09F00F0E0C6E01C10BF00C
:103AA00025EC09F0100E0C6E02C10BF025EC09F0AC
:103AB000110E0C6E03C10BF025EC09F00784010117
:103AC000B3EC20F057C100F158C101F107940A0E80
:103AD0000C6E00C10BF025EC09F00B0E0C6E01C151
:103AE0000BF025EC09F00C0E0C6E02C10BF025EC6E
:103AF00009F00D0E0C6E03C10BF025EC09F0C7EFB9
:103B00001DF007AAC7EF1DF007840101B3EC20F0F8
:103B100057C100F158C101F10794060E0C6E00C1A7
:103B20000BF025EC09F0070E0C6E01C10BF025EC33
:103B300009F0080E0C6E02C10BF025EC09F0090E1D
:103B40000C6E03C10BF025EC09F0078462C100F193
:103B500063C101F164C102F165C103F10794120E62
:103B60000C6E00C10BF025EC09F0130E0C6E01C1B8
:103B70000BF025EC09F0140E0C6E02C10BF025ECD5
:103B800009F0150E0C6E03C10BF025EC09F0079837
:103B9000079A0401805181197F0B0DE09EA8FED782
:103BA00014EE00F081517F0BE126E750812B0F01CD
:103BB000AD6EC9EF1DF0A4EF0AF018C100F119C1F4
:103BC00001F11AC102F11BC103F1000E046F000ED6
:103BD000056F010E066F000E076FE9EC1FF029A1BB
:103BE00008EF1EF02051D8B408EF1EF018C100F104
:103BF00019C101F11AC102F11BC103F1000E046FDA
:103C0000000E056F0A0E066F000E076FE9EC1FF03D
:103C10001200010104510013055101130651021352
:103C20000751031312000101186B196B1A6B1B6B00
:103C300012002AC182F40401300E82274DEC0BF0F1
:103C40002BC182F40401300E82274DEC0BF02CC105
:103C500082F40401300E82274DEC0BF02DC182F46A
:103C60000401300E82274DEC0BF02EC182F40401CA
:103C7000300E82274DEC0BF02FC182F40401300E80
:103C800082274DEC0BF030C182F40401300E822704
:103C90004DEC0BF031C182F40401300E82274DEC63
:103CA0000BF032C182F40401300E82274DEC0BF090
:103CB00033C182F40401300E82274DEC0BF0120068
:103CC0002FC182F40401300E82274DEC0BF030C17D
:103CD00082F40401300E82274DEC0BF031C182F4E6
:103CE0000401300E82274DEC0BF032C182F4040146
:103CF000300E82274DEC0BF033C182F40401300EFC
:103D000082274DEC0BF01200060E1F6E060E206E81
:103D1000060E216E1F2E8AEF1EF0202E8AEF1EF057
:103D2000212E8AEF1EF08B84020E1F6E020E206E73
:103D3000020E216E1F2E9AEF1EF0202E9AEF1EF01B
:103D4000212E9AEF1EF08B941200FF0E206E20C0E1
:103D500021F0030E1F6E8B841F2EABEF1EF0030E9F
:103D60001F6E212EABEF1EF08B9420C021F0030EAE
:103D70001F6E1F2EB9EF1EF0030E1F6E213EB9EF0E
:103D80001EF0202EA7EF1EF012000101005305E1E6
:103D9000015303E1025301E1002B88EC1FF0B3EC67
:103DA00020F03951006F3A51016F420E046F4B0EF3
:103DB000056F000E066F000E076FC9EC1FF000C103
:103DC00004F101C105F102C106F103C107F118C1F7
:103DD00000F119C101F11AC102F11BC103F107B2CF
:103DE000F6EF1EF0BDEC1FF0F8EF1EF0B8EC1FF080
:103DF00000C118F101C119F102C11AF103C11BF18F
:103E00001200B3EC20F059C100F15AC101F1060EC5
:103E10003CEC09F0E8CF04F1070E3CEC09F0E8CFE8
:103E200005F1080E3CEC09F0E8CF06F1090E3CEC78
:103E300009F0E8CF07F1B8EC1FF000C124F101C18F
:103E400025F102C126F103C127F1290E046F000EEE
:103E5000056F000E066F000E076FC9EC1FF0EE0E27
:103E6000046F430E056F000E066F000E076FBDEC6A
:103E70001FF024C104F125C105F126C106F127C1B7
:103E800007F1C9EC1FF000C11CF101C11DF102C115
:103E90001EF103C11FF1120E3CEC09F0E8CF04F152
:103EA000130E3CEC09F0E8CF05F1140E3CEC09F0E0
:103EB000E8CF06F1150E3CEC09F0E8CF07F10D0E46
:103EC000006F000E016F000E026F000E036FC9EC51
:103ED0001FF0180E046F000E056F000E066F000E27
:103EE000076FE9EC1FF01CC104F11DC105F11EC1F3
:103EF00006F11FC107F1BDEC1FF06A0E046F2A0E18
:103F0000056F000E066F000E076FB8EC1FF0120071
:103F1000BF0EFA6E200E3A6F396BD890003701371A
:103F200002370337D8B099EF1FF03A2F8EEF1FF00A
:103F300039073A070353D8B412000331070B80093D
:103F40003F6F03390F0B010F396F80EC5FF0406F4B
:103F5000390580EC5FF0405D405F396B3F33D8B08E
:103F6000392739333FA9AEEF1FF0405139271200EE
:103F70000101D8EC20F0D8B012000101035107195B
:103F8000346F9BEC20F0D8900751031934AF800FA9
:103F900012000101346BBFEC20F0D8A0D5EC20F06A
:103FA000D8B01200AAEC20F0B3EC20F01F0E366F50
:103FB000EBEC20F00B35D8B09BEC20F0D8A003350B
:103FC000D8B01200362FD8EF1FF034B1C2EC20F079
:103FD00012000101346B045105110611071100088C
:103FE000D8A0BFEC20F0D8A0D5EC20F0D8B01200BB
:103FF000086B096B0A6B0B6BEBEC20F01F0E366F36
:10400000EBEC20F007510B5DD8A413EF20F0065124
:104010000A5DD8A413EF20F00551095DD8A413EF71
:1040200020F00451085DD8A026EF20F00451085F6D
:104030000551D8A0053D095F0651D8A0063D0A5F8D
:104040000751D8A0073D0B5FD8900081362F00EFB5
:1040500020F034B1C2EC20F0346BBFEC20F0D890EB
:10406000EFEC20F007510B5DD8A443EF20F0065190
:104070000A5DD8A443EF20F00551095DD8A443EFB1
:1040800020F00451085DD8A052EF20F0003F52EF1D
:1040900020F0013F52EF20F0023F52EF20F0032BBF
:1040A000D8B4120034B1C2EC20F012000101346B1C
:1040B000BFEC20F0D8B01200F4EC20F0200E366FE8
:1040C000003701370237033711EE33F00A0E376F2E
:1040D000E7360A0EE75CD8B0E76EE552372F68EF97
:1040E00020F0362F60EF20F034B12981D8901200F3
:1040F00001010A0E346F200E366F11EE29F0345193
:10410000376F0A0ED890E652D8B0E726E732372F3D
:1041100083EF20F00333023301330033362F7DEF7A
:1041200020F0E750FF0FD8A00335D8B0120029B116
:10413000C2EC20F01200045100270551D8B0053D13
:1041400001270651D8B0063D02270751D8B0073DD8
:10415000032712000051086F0151096F02510A6FC5
:1041600003510B6F12000101006B016B026B036BBB
:1041700012000101046B056B066B076B120003351F
:10418000D8A012000351800B001F011F021F031F44
:10419000003FD2EF20F0013FD2EF20F0023FD2EFFC
:1041A00020F0032B342B032512000735D8A0120072
:1041B0000751800B041F051F061F071F043FE8EF70
:1041C00020F0053FE8EF20F0063FE8EF20F0072B56
:1041D000342B072512000037013702370337083721
:1041E00009370A370B3712000101296B2A6B2B6B39
:1041F0002C6B2D6B2E6B2F6B306B316B326B336BEB
:10420000120001012A510F0B2A6F2B510F0B2B6F3C
:104210002C510F0B2C6F2D510F0B2D6F2E510F0B9F
:104220002E6F2F510F0B2F6F30510F0B306F3151FD
:104230000F0B316F32510F0B326F33510F0B336F46
:10424000120000011750FF0A01E11200390EC86E7A
:10425000800EC76E280EC66E000EC56E1650000A80
:10426000D8B45CEF21F01650010AD8B475EF21F0F4
:104270001650020AD8B48EEF21F01650030AD8B4B3
:10428000A7EF21F01650040AD8B4CFEF21F0165052
:10429000050AD8B4E8EF21F01650060AD8B401EFA9
:1042A00022F01650070AD8B41AEF22F01650080A66
:1042B000D8B433EF22F012001750000AD8B452EFEE
:1042C00022F01750010AD8B456EF22F01750020A14
:1042D000D8B45AEF22F01750030AD8B45EEF22F098
:1042E0001750040AD8B4D1EF22F01750000AD8B4FE
:1042F00066EF22F01750010AD8B46AEF22F0175087
:10430000020AD8B46EEF22F01750030AD8B472EF45
:1043100022F01750040AD8B4D1EF22F01750000A47
:10432000D8B476EF22F01750010AD8B47AEF22F011
:104330001750020AD8B47EEF22F01750030AD8B4FF
:1043400082EF22F01750040AD8B4D1EF22F01750B0
:10435000000AD8B48FEF22F01750010AD8B493EFB7
:1043600022F01750020AD8B497EF22F01750030A30
:10437000D8B4ABEF22F01750040AD8B4AFEF22F054
:104380001750050AD8B4B3EF22F01750060AD8B474
:10439000B7EF22F01750070AD8B4BAEF22F017503F
:1043A000000AD8B4BEEF22F01750010AD8B4C2EF09
:1043B00022F01750020AD8B4C6EF22F01750030AB1
:1043C000D8B4CAEF22F01750040AD8B4CDEF22F0C7
:1043D0001750000AD8B4D5EF22F01750010AD8B40C
:1043E000D9EF22F01750020AD8B4DDEF22F01750AF
:1043F000030AD8B4E1EF22F01750040AD8B4D1EF81
:1044000022F01750000AD8B4EBEF22F01750010A3F
:10441000D8B4EFEF22F01750020AD8B4F3EF22F02D
:104420001750030AD8B4F7EF22F01750040AD8B493
:10443000D1EF22F01750000AD8B4F8EF22F017504D
:10444000010AD8B4FCEF22F01750020AD8B400EFEA
:1044500023F01750030AD8B404EF23F01750040ACE
:10446000D8B4D1EF22F01750000AD8B405EF23F0EA
:104470001750010AD8B409EF23F01750020AD8B434
:104480000DEF23F01750030AD8B411EF23F01750A3
:10449000040AD8B412EF23F01750050AD8B415EF68
:1044A00023F012009E96C580172A1200E20EC96EF4
:1044B000172A1200770EC96E172A1200020EE86E34
:1044C0008AB4E88AE8CFC9FF172A12009E96C580F1
:1044D000172A1200E20EC96E172A1200790EC96E51
:1044E000172A1200000EC96E172A12009E96C58068
:1044F000172A1200E20EC96E172A12007A0EC96E30
:10450000172A120019BC03D0DEC1E8FF04D01950ED
:10451000E844E8441F09E8CFC9FF172A12009E9615
:10452000C580172A1200E20EC96E172A120011BAAE
:1045300003D011BC01D003D0050E166E3ED0010190
:10454000DA67A7EF22F0100EC96EA9EF22F0DAC1E8
:10455000C9FF172A1200DBC1C9FF172A1200DCC1EC
:10456000C9FF172A1200DDC1C9FF172A1200C5842E
:10457000172A1200FF0E176E1E9E12009E96C5800F
:10458000172A1200E20EC96E172A1200760EC96EA3
:10459000172A1200C584172A1200FF0E176E1E9EDE
:1045A0001200C584162A176A12009E96C580172A23
:1045B0001200E20EC96E172A12007B0EC96E172A6E
:1045C000120011AA04D0230EC96E172A12001C0E65
:1045D000C96E172A12009E96C580172A1200E20E95
:1045E000C96E172A12007C0EC96E172A1200E9D76D
:1045F0009E96C580172A1200E20EC96E172A120075
:104600007D0EC96E172A1200DCD79E96C580172A28
:104610001200E20EC96E172A12007E0EC96E172A0A
:104620001200CFD7C584172A1200FF0E176E1E9EE8
:1046300012001750FF0AD8B4D7EF23F0390EC86E16
:10464000800EC76E280EC66E000EC56E1650000A8C
:10465000D8B432EF23F01650010AD8B446EF23F055
:10466000D7EF23F01750000AD8B484EF23F0175087
:10467000010AD8B488EF23F01750020AD8B492EF99
:1046800023F01750030AD8B495EF23F01750000A0F
:10469000D8B49BEF23F01750010AD8B49FEF23F052
:1046A0001750020AD8B4A9EF23F01750030AD8B460
:1046B000ACEF23F01750040AD8B4B2EF23F0175030
:1046C000050AD8B4B5EF23F01750060AD8B4BBEFEB
:1046D00023F01750070AD8B4BEEF23F01750080A8A
:1046E000D8B4C4EF23F01750090AD8B4C7EF23F0A9
:1046F00017500A0AD8B4CDEF23F017500B0AD8B4DC
:10470000D0EF23F0D7EF23F09E96C580D6EF23F0AD
:1047100018B004D04E0EC96ED6EF23F0500EC96EFD
:10472000D6EF23F0C584D6EF23F0162AFF0E176EBE
:104730001280D7EF23F09E96C580D6EF23F018B0F5
:1047400004D04F0EC96ED6EF23F0510EC96ED6EFCE
:1047500023F0C586D6EF23F0C9CF25F0C59AC588CA
:10476000D6EF23F0C586D6EF23F0C9CF26F0C59A41
:10477000C588D6EF23F0C586D6EF23F0C9CF27F042
:10478000C59AC588D6EF23F0C586D6EF23F0C9CFEA
:1047900028F0C58AC588D6EF23F0C584D6EF23F06C
:1047A000FF0E176E12861E9CD7EF23F0172A1200F9
:1047B00012B012D012B213D012B414D012A612003A
:1047C00007B01200129625C029F026C02AF027C093
:1047D0002BF028C02CF012001290128212001292BC
:1047E0001284120000011750FF0A04E11294176AA4
:0647F00019EC23F0120099
:10BF0000E844F926000C160C2B0C3F0C520C640C68
:10BF1000760C860C960CA50CB30CC10CCF0CDC0C6B
:06BF2000E80CF40C000C1B
:00000001FF
